Archive member included because of file (symbol)

c:/program files/yagarto/bin/../lib/gcc/arm-elf/4.3.3\libgcc.a(_udivsi3.o)
                              ../common/src/rprintf.o (__udivsi3)
c:/program files/yagarto/bin/../lib/gcc/arm-elf/4.3.3\libgcc.a(_umodsi3.o)
                              ../common/src/rprintf.o (__umodsi3)
c:/program files/yagarto/bin/../lib/gcc/arm-elf/4.3.3\libgcc.a(_dvmd_tls.o)
                              c:/program files/yagarto/bin/../lib/gcc/arm-elf/4.3.3\libgcc.a(_udivsi3.o) (__div0)

Allocating common symbols
Common symbol       size              file

sp                  0x4               Sound.o
s                   0x14              Sound.o

Memory Configuration

Name             Origin             Length             Attributes
flash            0x00000000         0x00080000
ram_isp_low      0x40000120         0x000000df         a
ram              0x40000200         0x00007f01
ram_isp_high     0x40007fe0         0x00000020         a
ram_usb_dma      0x7fd00000         0x00002000
*default*        0x00000000         0xffffffff

Linker script and memory map

LOAD ../common/src/crt.o
LOAD ../common/src/startup.o
LOAD ../common/src/armVIC.o
LOAD ../common/src/TFT018.o
LOAD ../common/src/rprintf.o
LOAD Sound.o
LOAD Data.o
START GROUP
LOAD c:/program files/yagarto/bin/../lib/gcc/arm-elf/4.3.3\libgcc.a
LOAD c:/program files/yagarto/bin/../lib/gcc/arm-elf/4.3.3/../../../../arm-elf/lib\libc.a
END GROUP
                0x40007edc                _stack_end = 0x40007edc
                0x00000000                . = 0x0

startup
 *(.startup)

.text           0x00000000     0x48ec
 *(.text)
 .text          0x00000000       0xd8 ../common/src/crt.o
                0x00000000                _startup
                0x00000040                Reset_Handler
 .text          0x000000d8       0x84 ../common/src/startup.o
                0x000000e4                UNDEF_Routine
                0x000000e0                SWI_Routine
                0x000000dc                FIQ_Routine
                0x000000d8                IRQ_Routine
                0x000000e8                Initialize
 .text          0x0000015c       0x78 ../common/src/armVIC.o
                0x0000016c                restoreIRQ
                0x000001c4                enableFIQ
                0x00000198                disableFIQ
                0x00000188                enableIRQ
                0x000001a8                restoreFIQ
                0x0000015c                disableIRQ
 .text          0x000001d4      0xaf4 ../common/src/TFT018.o
                0x000002f8                LCD_Reg_Set
                0x000004cc                LCD_SetArea
                0x00000aec                LCD_PutString
                0x00000614                LCD_Clear_Screen
                0x0000052c                LCD_Rectangle
                0x00000b90                LCD_BMP
                0x00000810                LCD_PutChar8x8
                0x000001d4                BacklightOn
                0x0000063c                LCD_SetPixel
                0x00000290                LCD_Bus_Write_Data
                0x00000378                LCD_Init
                0x00000940                LCD_PutChar
                0x00000234                LCD_Bus_Initial
                0x000006dc                LCD_PutChar8x16
                0x00000c90                LCD_Bus_Read_Pixel
                0x000002d4                LCD_Bus_Read_Byte
                0x00000230                Delay1Ms
                0x00000264                LCD_Bus_Write_Byte
                0x00000978                PutGB1616
 .text          0x00000cc8      0x258 ../common/src/rprintf.o
                0x00000cc8                rprintf_devopen
                0x00000d0c                rprintf
 .text          0x00000f20      0x27c Sound.o
                0x0000100c                input_str
                0x00001030                main
 .text          0x0000119c        0x0 Data.o
 .text          0x0000119c      0x110 c:/program files/yagarto/bin/../lib/gcc/arm-elf/4.3.3\libgcc.a(_udivsi3.o)
                0x0000119c                __udivsi3
                0x0000119c                __aeabi_uidiv
                0x00001294                __aeabi_uidivmod
 .text          0x000012ac       0xcc c:/program files/yagarto/bin/../lib/gcc/arm-elf/4.3.3\libgcc.a(_umodsi3.o)
                0x000012ac                __umodsi3
 .text          0x00001378        0x4 c:/program files/yagarto/bin/../lib/gcc/arm-elf/4.3.3\libgcc.a(_dvmd_tls.o)
                0x00001378                __aeabi_ldiv0
                0x00001378                __div0
                0x00001378                __aeabi_idiv0
 *(.rodata)
 .rodata        0x0000137c     0x1248 ../common/src/TFT018.o
                0x00002384                codeGB_16
                0x00001b7c                Font8x8
                0x0000137c                Font8x16
 .rodata        0x000025c4     0x2304 Data.o
                0x000025c4                SoundData
                0x000048c4                SoundCount
 *(.rodata*)
 .rodata.str1.1
                0x000048c8       0x22 Sound.o
 *(.glue_7)
 *fill*         0x000048ea        0x2 00
 .glue_7        0x000048ec        0x0 ../common/src/crt.o
 .glue_7        0x000048ec        0x0 ../common/src/startup.o
 .glue_7        0x000048ec        0x0 ../common/src/armVIC.o
 .glue_7        0x000048ec        0x0 ../common/src/TFT018.o
 .glue_7        0x000048ec        0x0 ../common/src/rprintf.o
 .glue_7        0x000048ec        0x0 Sound.o
 .glue_7        0x000048ec        0x0 Data.o
 .glue_7        0x000048ec        0x0 c:/program files/yagarto/bin/../lib/gcc/arm-elf/4.3.3\libgcc.a(_udivsi3.o)
 .glue_7        0x000048ec        0x0 c:/program files/yagarto/bin/../lib/gcc/arm-elf/4.3.3\libgcc.a(_umodsi3.o)
 .glue_7        0x000048ec        0x0 c:/program files/yagarto/bin/../lib/gcc/arm-elf/4.3.3\libgcc.a(_dvmd_tls.o)
 *(.glue_7t)
 .glue_7t       0x000048ec        0x0 ../common/src/crt.o
 .glue_7t       0x000048ec        0x0 ../common/src/startup.o
 .glue_7t       0x000048ec        0x0 ../common/src/armVIC.o
 .glue_7t       0x000048ec        0x0 ../common/src/TFT018.o
 .glue_7t       0x000048ec        0x0 ../common/src/rprintf.o
 .glue_7t       0x000048ec        0x0 Sound.o
 .glue_7t       0x000048ec        0x0 Data.o
 .glue_7t       0x000048ec        0x0 c:/program files/yagarto/bin/../lib/gcc/arm-elf/4.3.3\libgcc.a(_udivsi3.o)
 .glue_7t       0x000048ec        0x0 c:/program files/yagarto/bin/../lib/gcc/arm-elf/4.3.3\libgcc.a(_umodsi3.o)
 .glue_7t       0x000048ec        0x0 c:/program files/yagarto/bin/../lib/gcc/arm-elf/4.3.3\libgcc.a(_dvmd_tls.o)
                0x000048ec                _etext = .

.vfp11_veneer   0x40000120        0x0
 .vfp11_veneer  0x40000120        0x0 ../common/src/crt.o
 .vfp11_veneer  0x40000120        0x0 ../common/src/startup.o
 .vfp11_veneer  0x40000120        0x0 ../common/src/armVIC.o
 .vfp11_veneer  0x40000120        0x0 ../common/src/TFT018.o
 .vfp11_veneer  0x40000120        0x0 ../common/src/rprintf.o
 .vfp11_veneer  0x40000120        0x0 Sound.o
 .vfp11_veneer  0x40000120        0x0 Data.o
 .vfp11_veneer  0x40000120        0x0 c:/program files/yagarto/bin/../lib/gcc/arm-elf/4.3.3\libgcc.a(_udivsi3.o)
 .vfp11_veneer  0x40000120        0x0 c:/program files/yagarto/bin/../lib/gcc/arm-elf/4.3.3\libgcc.a(_umodsi3.o)
 .vfp11_veneer  0x40000120        0x0 c:/program files/yagarto/bin/../lib/gcc/arm-elf/4.3.3\libgcc.a(_dvmd_tls.o)

.v4_bx          0x40000120        0x0
 .v4_bx         0x40000120        0x0 ../common/src/crt.o
 .v4_bx         0x40000120        0x0 ../common/src/startup.o
 .v4_bx         0x40000120        0x0 ../common/src/armVIC.o
 .v4_bx         0x40000120        0x0 ../common/src/TFT018.o
 .v4_bx         0x40000120        0x0 ../common/src/rprintf.o
 .v4_bx         0x40000120        0x0 Sound.o
 .v4_bx         0x40000120        0x0 Data.o
 .v4_bx         0x40000120        0x0 c:/program files/yagarto/bin/../lib/gcc/arm-elf/4.3.3\libgcc.a(_udivsi3.o)
 .v4_bx         0x40000120        0x0 c:/program files/yagarto/bin/../lib/gcc/arm-elf/4.3.3\libgcc.a(_umodsi3.o)
 .v4_bx         0x40000120        0x0 c:/program files/yagarto/bin/../lib/gcc/arm-elf/4.3.3\libgcc.a(_dvmd_tls.o)

.data           0x40000200        0x0 load address 0x000048ec
                0x40000200                _data = .
 *(.data)
 .data          0x40000200        0x0 ../common/src/crt.o
 .data          0x40000200        0x0 ../common/src/startup.o
 .data          0x40000200        0x0 ../common/src/armVIC.o
 .data          0x40000200        0x0 ../common/src/TFT018.o
 .data          0x40000200        0x0 ../common/src/rprintf.o
 .data          0x40000200        0x0 Sound.o
 .data          0x40000200        0x0 Data.o
 .data          0x40000200        0x0 c:/program files/yagarto/bin/../lib/gcc/arm-elf/4.3.3\libgcc.a(_udivsi3.o)
 .data          0x40000200        0x0 c:/program files/yagarto/bin/../lib/gcc/arm-elf/4.3.3\libgcc.a(_umodsi3.o)
 .data          0x40000200        0x0 c:/program files/yagarto/bin/../lib/gcc/arm-elf/4.3.3\libgcc.a(_dvmd_tls.o)
                0x40000200                _edata = .

.bss            0x40000200       0x28
                0x40000200                _bss_start = .
 *(.bss)
 .bss           0x40000200        0x0 ../common/src/crt.o
 .bss           0x40000200        0x0 ../common/src/startup.o
 .bss           0x40000200        0x0 ../common/src/armVIC.o
 .bss           0x40000200        0x1 ../common/src/TFT018.o
                0x40000200                Font
 *fill*         0x40000201        0x3 00
 .bss           0x40000204        0x4 ../common/src/rprintf.o
 .bss           0x40000208        0x8 Sound.o
                0x40000208                Index
                0x4000020c                Volume
 .bss           0x40000210        0x0 Data.o
 .bss           0x40000210        0x0 c:/program files/yagarto/bin/../lib/gcc/arm-elf/4.3.3\libgcc.a(_udivsi3.o)
 .bss           0x40000210        0x0 c:/program files/yagarto/bin/../lib/gcc/arm-elf/4.3.3\libgcc.a(_umodsi3.o)
 .bss           0x40000210        0x0 c:/program files/yagarto/bin/../lib/gcc/arm-elf/4.3.3\libgcc.a(_dvmd_tls.o)
 COMMON         0x40000210       0x18 Sound.o
                0x40000210                sp
                0x40000214                s
                0x40000228                . = ALIGN (0x4)
                0x40000228                _bss_end = .
                0x40000228                _end = .
OUTPUT(Sound.elf elf32-littlearm)

.ARM.attributes
                0x00000000       0x10
 .ARM.attributes
                0x00000000       0x10 ../common/src/crt.o
 .ARM.attributes
                0x00000010       0x10 ../common/src/startup.o
 .ARM.attributes
                0x00000020       0x10 ../common/src/armVIC.o
 .ARM.attributes
                0x00000030       0x10 ../common/src/TFT018.o
 .ARM.attributes
                0x00000040       0x10 ../common/src/rprintf.o
 .ARM.attributes
                0x00000050       0x10 Sound.o
 .ARM.attributes
                0x00000060       0x10 Data.o
 .ARM.attributes
                0x00000070       0x10 c:/program files/yagarto/bin/../lib/gcc/arm-elf/4.3.3\libgcc.a(_udivsi3.o)
 .ARM.attributes
                0x00000080       0x10 c:/program files/yagarto/bin/../lib/gcc/arm-elf/4.3.3\libgcc.a(_umodsi3.o)
 .ARM.attributes
                0x00000090       0x10 c:/program files/yagarto/bin/../lib/gcc/arm-elf/4.3.3\libgcc.a(_dvmd_tls.o)

.debug_abbrev   0x00000000      0x704
 .debug_abbrev  0x00000000       0x69 ../common/src/startup.o
 .debug_abbrev  0x00000069       0xea ../common/src/armVIC.o
 .debug_abbrev  0x00000153      0x2bd ../common/src/TFT018.o
 .debug_abbrev  0x00000410      0x140 ../common/src/rprintf.o
 .debug_abbrev  0x00000550      0x10a Sound.o
 .debug_abbrev  0x0000065a       0x6e Data.o
 .debug_abbrev  0x000006c8       0x14 c:/program files/yagarto/bin/../lib/gcc/arm-elf/4.3.3\libgcc.a(_udivsi3.o)
 .debug_abbrev  0x000006dc       0x14 c:/program files/yagarto/bin/../lib/gcc/arm-elf/4.3.3\libgcc.a(_umodsi3.o)
 .debug_abbrev  0x000006f0       0x14 c:/program files/yagarto/bin/../lib/gcc/arm-elf/4.3.3\libgcc.a(_dvmd_tls.o)

.debug_info     0x00000000     0x13a7
 .debug_info    0x00000000       0xb4 ../common/src/startup.o
 .debug_info    0x000000b4      0x2bc ../common/src/armVIC.o
 .debug_info    0x00000370      0xa85 ../common/src/TFT018.o
 .debug_info    0x00000df5      0x207 ../common/src/rprintf.o
 .debug_info    0x00000ffc      0x178 Sound.o
 .debug_info    0x00001174       0x77 Data.o
 .debug_info    0x000011eb       0x94 c:/program files/yagarto/bin/../lib/gcc/arm-elf/4.3.3\libgcc.a(_udivsi3.o)
 .debug_info    0x0000127f       0x94 c:/program files/yagarto/bin/../lib/gcc/arm-elf/4.3.3\libgcc.a(_umodsi3.o)
 .debug_info    0x00001313       0x94 c:/program files/yagarto/bin/../lib/gcc/arm-elf/4.3.3\libgcc.a(_dvmd_tls.o)

.debug_line     0x00000000      0x70f
 .debug_line    0x00000000       0x77 ../common/src/startup.o
 .debug_line    0x00000077       0x75 ../common/src/armVIC.o
 .debug_line    0x000000ec      0x32c ../common/src/TFT018.o
 .debug_line    0x00000418       0xd6 ../common/src/rprintf.o
 .debug_line    0x000004ee       0x7b Sound.o
 .debug_line    0x00000569       0x27 Data.o
 .debug_line    0x00000590       0x96 c:/program files/yagarto/bin/../lib/gcc/arm-elf/4.3.3\libgcc.a(_udivsi3.o)
 .debug_line    0x00000626       0x7f c:/program files/yagarto/bin/../lib/gcc/arm-elf/4.3.3\libgcc.a(_umodsi3.o)
 .debug_line    0x000006a5       0x6a c:/program files/yagarto/bin/../lib/gcc/arm-elf/4.3.3\libgcc.a(_dvmd_tls.o)

.debug_frame    0x00000000      0x3d0
 .debug_frame   0x00000000       0x60 ../common/src/startup.o
 .debug_frame   0x00000060       0x70 ../common/src/armVIC.o
 .debug_frame   0x000000d0      0x1e0 ../common/src/TFT018.o
 .debug_frame   0x000002b0       0x6c ../common/src/rprintf.o
 .debug_frame   0x0000031c       0x64 Sound.o
 .debug_frame   0x00000380       0x28 c:/program files/yagarto/bin/../lib/gcc/arm-elf/4.3.3\libgcc.a(_udivsi3.o)
 .debug_frame   0x000003a8       0x28 c:/program files/yagarto/bin/../lib/gcc/arm-elf/4.3.3\libgcc.a(_umodsi3.o)

.debug_pubnames
                0x00000000      0x30f
 .debug_pubnames
                0x00000000       0x63 ../common/src/startup.o
 .debug_pubnames
                0x00000063       0x6a ../common/src/armVIC.o
 .debug_pubnames
                0x000000cd      0x196 ../common/src/TFT018.o
 .debug_pubnames
                0x00000263       0x32 ../common/src/rprintf.o
 .debug_pubnames
                0x00000295       0x4b Sound.o
 .debug_pubnames
                0x000002e0       0x2f Data.o

.debug_aranges  0x00000000      0x100
 .debug_aranges
                0x00000000       0x20 ../common/src/startup.o
 .debug_aranges
                0x00000020       0x20 ../common/src/armVIC.o
 .debug_aranges
                0x00000040       0x20 ../common/src/TFT018.o
 .debug_aranges
                0x00000060       0x20 ../common/src/rprintf.o
 .debug_aranges
                0x00000080       0x20 Sound.o
 .debug_aranges
                0x000000a0       0x20 c:/program files/yagarto/bin/../lib/gcc/arm-elf/4.3.3\libgcc.a(_udivsi3.o)
 .debug_aranges
                0x000000c0       0x20 c:/program files/yagarto/bin/../lib/gcc/arm-elf/4.3.3\libgcc.a(_umodsi3.o)
 .debug_aranges
                0x000000e0       0x20 c:/program files/yagarto/bin/../lib/gcc/arm-elf/4.3.3\libgcc.a(_dvmd_tls.o)

.debug_ranges   0x00000000      0x7a8
 .debug_ranges  0x00000000       0x30 ../common/src/startup.o
 .debug_ranges  0x00000030      0x760 ../common/src/TFT018.o
 .debug_ranges  0x00000790       0x18 ../common/src/rprintf.o

.debug_str      0x00000000      0x3ae
 .debug_str     0x00000000       0x8b ../common/src/startup.o
 .debug_str     0x0000008b       0x9d ../common/src/armVIC.o
                                 0xf3 (size before relaxing)
 .debug_str     0x00000128      0x18e ../common/src/TFT018.o
                                0x1f7 (size before relaxing)
 .debug_str     0x000002b6       0xbe ../common/src/rprintf.o
                                0x180 (size before relaxing)
 .debug_str     0x00000374       0x33 Sound.o
                                 0xde (size before relaxing)
 .debug_str     0x000003a7        0x7 Data.o
                                 0x52 (size before relaxing)

.comment        0x00000000       0x6c
 .comment       0x00000000       0x12 ../common/src/startup.o
 .comment       0x00000012       0x12 ../common/src/armVIC.o
 .comment       0x00000024       0x12 ../common/src/TFT018.o
 .comment       0x00000036       0x12 ../common/src/rprintf.o
 .comment       0x00000048       0x12 Sound.o
 .comment       0x0000005a       0x12 Data.o

.debug_loc      0x00000000      0xc09
 .debug_loc     0x00000000       0x72 ../common/src/armVIC.o
 .debug_loc     0x00000072      0x927 ../common/src/TFT018.o
 .debug_loc     0x00000999      0x1ea ../common/src/rprintf.o
 .debug_loc     0x00000b83       0x86 Sound.o
